:100000000C9415010C943D010C943D010C943D01A0
:100010000C943D010C943D010C943D010C943D0168
:100020000C943D010C943D010C943D010C943D0158
:100030000C943D010C943D010C943D010C943D0148
:100040000C94BD1A0C943D010C944E1D0C94801D13
:100050000C943D010C943D010C943D010C943D0128
:100060000C940B170C943D017A127F1282128F129E
:10007000931299129B12C312C612CD12E012084AB3
:10008000D73B3BCE016E84BCBFFDC12F3D6C7431AC
:100090009ABD56833DDA3D00C77F11BED9E4BB4C03
:1000A0003E916BAAAABE000000803F05A84CCDB2CD
:1000B000D44EB93836A9020C50B9918688083CA6AE
:1000C000AAAA2ABE000000803F07634236B79BD829
:1000D000A71A39685618AEBAAB558C1D3CB7CC5729
:1000E00063BD6DEDFD753EF6177231BF00000080F7
:1000F0003F08000000BE922449123EABAAAA2ABEC5
:10010000CDCCCC4C3E00000080BEABAAAAAA3E00DB
:10011000000000BF000000803F0000000000084118
:1001200078D3BB4387D1133D190E3CC3BD4282AD8A
:100130002B3E68EC8276BED98FE1A93E4C80EFFF62
:10014000BE01C4FF7F3F0000000000004D50553647
:1001500030353020636F6E6E656374696F6E206634
:1001600061696C6564004D50553630353020636FE1
:100170006E6E656374696F6E207375636365737308
:1001800066756C0054657374696E67206465766982
:10019000636520636F6E6E656374696F6E732E2E78
:1001A0002E00496E697469616C697A696E672049CD
:1001B000324320646576696365732E2E2E002050CD
:1001C0006978656C73203D2000436F756E74203D27
:1001D00020000000000800020100000304070000E6
:1001E000000000000000010204081020408001020D
:1001F000040810200102040810200404040404046C
:1002000004040202020202020303030303030000C8
:100210000000250028002B0000000000240027001B
:100220002A00420C2916B01D500C11241FBECFEF1E
:10023000D8E0DEBFCDBF11E0A0E0B1E0EAEFF1E52C
:1002400002C005900D92A83AB107D9F724E0A8EAB8
:10025000B1E001C01D92AE3DB207E1F712E0C8E285
:10026000D2E004C02297FE010E946724C232D10767
:10027000C9F70E94F41D0C94F0280C94000061153D
:10028000710581F0DB010D900020E9F7AD014150CF
:100290005109461B570BDC01ED91FC910280F38163
:1002A000E02D099480E090E00895CF92DF92EF92E4
:1002B000FF92CF93DF9326E040E056E960E070E0E4
:1002C0008DE394E00E94EC1C89EB91E00E944A13BC
:1002D000109280008FE08093810010928500109230
:1002E000840089EB91E00E94CE138091840090916C
:1002F00085000C9668E170E00E94FC238CE390E09E
:10030000861B970B90930B0180930A0169EC71E0B7
:100310008DE394E00E942B1E609184007091850013
:100320004AE050E08DE394E00E94351F6EEB71E0EF
:100330008DE394E00E942B1E60910A0170910B01E5
:100340004AE050E08DE394E00E94101F84E793E0C0
:100350000E94EF1562EA71E08DE394E00E945B1E5B
:100360008AEA91E00E94851A64E871E08DE394E0E6
:100370000E945B1E8AEA91E00E94B51A80935303A3
:10038000882319F066E671E002C06CE471E08DE349
:1003900094E00E945B1E61E08DE00E949A1B0E9427
:1003A000071B6093CE017093CF018093D00190938F
:1003B000D10160934F037093500380935103909346
:1003C0005203C0910A01D0910B01EBEDF1E020E066
:1003D00030E081E090E0A0E0B0E0C831D1051CF051
:1003E00043E050E002C042E050E02417350754F4E7
:1003F00011821082868B978BA08FB18F2F5F3F4F1A
:100400007A96EBCFBE01660F771F6C0F7D1F882792
:1004100077FD8095982F0E94E4206B017C019B0161
:10042000AC010E947C1FA70196010E94FD216B0177
:100430007C0188EC8C9FB0018D9F700D1124882762
:1004400077FD8095982F0E94E42020ED3FE049E45D
:1004500050E40E9449209B01AC01C701B6010E94F3
:100460007C1F6093430270934402809345029093F3
:1004700046021092470210924802109249021092CE
:100480004A0281E090E09093D6018093D501DF91FC
:10049000CF91FF90EF90DF90CF9008951F93CF936F
:1004A000DF939C013327E62FF0E02535310544F535
:1004B000A901440F551F420F531F4E9FC0014F9F6C
:1004C000900D5E9F900D1124CFEFD0E0BE010E94F1
:1004D0001024462F5DEF5203C001539F900D11244D
:1004E0009C0121503F4F2E9FC0012F9F900D3E9F9A
:1004F000900D1124BE010E941024862F60E054C08C
:100500002A3A310544F5255531096DEF6203A00102
:10051000639F500D112441505F4F4E9FC0014F9F6C
:10052000900D5E9F900D1124CFEFD0E0BE010E9490
:100530001024462FD901AA0FBB1FA20FB31FAE9FD5
:10054000C001AF9F900DBE9F900D1124BE010E946F
:10055000102480E029C02A5A31096DEF6203A001FE
:10056000639F500D112441505F4F4E9FC0014F9F1C
:10057000900D5E9F900D1124CFEFD0E0BE010E9440
:100580001024162FA901440F551F420F531F4E9FD1
:10059000C0014F9F900D5E9F900D1124BE010E94DF
:1005A0001024862F40E0612FDF91CF911F910C9492
:1005B0004F154F925F926F927F928F929F92AF9260
:1005C000BF92CF92DF92EF92FF920F931F93CF9340
:1005D000DF93A42FB0E0A80FB11D2D01662457FCB6
:1005E0006094762C032F10E0070F111D4801AA24F8
:1005F00097FCA094BA2CC22FD0E0C60FD11D9E014B
:10060000442737FD4095542F91E06FEF4616510473
:100610006104710409F008F490E081E06FEF861640
:100620009104A104B10409F008F480E0892B31F4AD
:100630002F3F31054105510549F140F17301620138
:10064000C80CD91CEA1CFB1CC20ED31EE41EF51EEE
:100650002FEF30E00E947A24A70196010E94242403
:1006600029013A012FEF30E0D8010E947A24A70136
:1006700096010E94242449015A012FEF30E0DE0147
:100680000E947A24A70196010E942424C2017727A0
:100690006627BA2CA92C982C8824682979298A29BC
:1006A0009B29622B732B842B952BDF91CF911F916C
:1006B0000F91FF90EF90DF90CF90BF90AF909F9001
:1006C0008F907F906F905F904F9008952F923F9200
:1006D0004F925F926F927F928F929F92AF92BF9252
:1006E000CF92DF92EF92FF920F931F93CF93DF93FE
:1006F000CDB7DEB7AC970FB6F894DEBF0FBECDBF57
:100700006091D40181E068276093D4018DE00E945C
:10071000D31B0E94071BC0906803D0906903E09030
:100720006A03F0906B03C982DA82EB82FC828090CC
:100730006C0390906D03A0906E03B0906F03A701BF
:1007400096015058C501B40190580E94EF1F6B01EB
:100750007C0160910A0170910B01882777FD8095DB
:10076000982F0E94E4202B013C019B01AC01C701A2
:10077000B6010E94FD2120ED3FE049EC50E40E94CB
:1007800049206B017C0120E030E0A9010E94422059
:1007900087FD09C0C0924B02D0924C02E0924D02FC
:1007A000F0924E020EC0A3019201C701B6010E9451
:1007B0007C1F60934B0270934C0280934D02909388
:1007C0004E02C501B4010E94F4226B017C016981D3
:1007D0007A818B819C810E94F4224B015C019B01F8
:1007E000AC01C701B6010E947C1F2B013C01609146
:1007F00064037091650380916603909167030E9482
:10080000F4226B017C01A50194010E947C1FA701C9
:1008100096010E947C1F9B01AC01C301B2010E94A2
:1008200049200E94B62220E030E048E452E40E94D1
:10083000FD216D837E838F8398870E94071B6B0148
:100840007C018091D7019091D801A091D901B091FC
:10085000DA01A7019601281B390B4A0B5B0BCA0171
:10086000B9010E94E22020E030E04AE754E40E940F
:1008700049206F8B788F898F9A8FC092D701D09241
:10088000D801E092D901F092DA01C0904702D090ED
:100890004802E0904902F0904A0260914302709150
:1008A0004402809145029091460220910A013091C4
:1008B0000B01283131052CF020E030E040E450E419
:1008C00004C020E030E040E050E40E94FD219B01A4
:1008D000AC01C701B6010E94422087FD12C01092F0
:1008E0004702109248021092490210924A024BEDC0
:1008F00051E05C874B8700E010E064E0262E312C4D
:1009000056C02BED622E21E0722EE12CF12C4424F6
:100910004394512C4EE1D42E52EEC52E80910A0103
:1009200090910B0148971CF083E090E002C082E0B8
:1009300090E0E816F9069CF6D3018D919C911197F1
:10094000892BB9F456968D919D910D90BC91A02D57
:10095000892B8A2B8B2B69F00E94071BF301868859
:100960009788A08CB18C681579058A059B0508F0DD
:100970001BC7FFEFEF1AFF0A1AE1610E711CCECF01
:1009800022E030E0021713070CF0DFC1AB85BC8515
:100990006D917C91615071096230710590F00F5F2B
:1009A0001F4F2B853C85265E3F4F3C872B878091D0
:1009B0000A0190910B018831910514F323E030E096
:1009C000E1CFBC01882777FD8095982F0E94E42015
:1009D0002B013C01EB85FC852285338544855585BB
:1009E00060914B0270914C0280914D0290914E02A9
:1009F0000E947B1F9B01AC010E947C1F20ED3FE009
:100A000049E450E40E94FD21A30192010E94492083
:100A10000E94AC229B01AC016D817E818F81988503
:100A20000E94FD214B015C01AB85BC8516962D9182
:100A30003D914D915C9119976F89788D898D9A8D33
:100A40000E94FD21EB85FC8566877787808B918BE3
:100A500022853385448555850E947C1F6B017C016E
:100A6000AB85BC851A966D937D938D939C931D9752
:100A700020E030E0A9010E94422087FF16C060916B
:100A80000A0170910B01882777FD8095982F0E94AD
:100A9000E4209B01AC01C701B6010E947C1FEB85DD
:100AA000FC856287738784879587AB85BC851A969A
:100AB000CD90DD90ED90FC901D97A3019201C701B0
:100AC000B6010E94F221181664F4A3019201C70135
:100AD000B6010E947B1FEB85FC8562877387848744
:100AE00095872F89388D498D5A8DC501B4010E9493
:100AF000FD21AB85BC8516962D913D914D915C9164
:100B000019970E947C1F6B017C0120E030E0A90155
:100B10000E94F2212DEC3CEC4CE45DE318161CF431
:100B2000C701B60103C0C701B60190580E94FD215C
:100B300069837A838B839C83EB85FC858280938099
:100B4000A480B5802BEA3AEA4AEA5EE3C501B40123
:100B50000E9460226B8B7C8B8D8B9E8B2F89388DB6
:100B6000498D5A8D69817A818B819C810E94FD21FA
:100B70002B893C894D895E890E9449209B01AC01EB
:100B800060E070E080E89FE30E947B1F9B01AC0166
:100B9000C701B6010E94FD216B017C01AB85BC85BC
:100BA00016966D937D938D939C9319971A962D911C
:100BB0003D914D915C911D9760914B0270914C025B
:100BC00080914D0290914E020E947B1F9B01AC01CF
:100BD0000E947C1F20ED3FE049E450E40E94FD218B
:100BE000A30192010E9449200E94462069837A83D2
:100BF0008B839C8320E030E040E05FE3C501B401DB
:100C00000E94FD21A70196010E94FD21A7019601E6
:100C10000E94FD216B017C01A50194016D817E8103
:100C20008F8198850E94FD214B015C0129813A81C9
:100C30004B815C8160E070E080E89FE30E947B1F55
:100C40009B01AC01C501B4010E94FD21A3019201E9
:100C50000E94FD2120ED3FE049EC50E40E94492034
:100C60009B01AC01C701B6010E947C1F6B017C0196
:100C7000EB85FC85628B738B848B958B9B01AC0120
:100C800060914702709148028091490290914A0216
:100C90000E947C1F60934702709348028093490230
:100CA00090934A02AB85BC858D919C9181309105D2
:100CB00029F520E030E040EA51E4C701B6010E9486
:100CC000422087FF6CCEEB85FC8511821082128258
:100CD0001382148215820E94071B6B017C012CED8C
:100CE00035E040E050E064EF71E080E090E00E9489
:100CF0005F1F6C0D7D1D8E1D9F1D20C0029709F08A
:100D00004ECE20E030E046E954E4C701B6010E942F
:100D1000422087FF44CEAB85BC8511963C922E9233
:100D2000C12CD12C90E8E92E9FEBF92E1296CD9292
:100D3000DD92ED92FC9215970E94071BEB85FC85D6
:100D4000668B778B808F918F2ACE4BED51E05CA71D
:100D50004BA71C8A1B8A80910A0190910B0148972E
:100D60001CF082E090E002C081E090E0CB88DC885B
:100D7000C816D9060CF0B5C26B897C896F5F7F4FAE
:100D80007C8B6B8B8BA59CA54A969AA789A71C0187
:100D900078A36F8F00910A0110910B0108311105A2
:100DA0001CF083E090E002C082E090E0CF8CD8A0FD
:100DB000C816D9060CF090C2ABA5BCA51296CD9072
:100DC000DD90ED90FC901597C982DA82EB82FC826F
:100DD00020E030E0A901C701B6010E9442201816A8
:100DE0000CF070C2D1011296CD90DD90ED90FC9088
:100DF0001597CD82DE82EF82F88620E030E0A901EF
:100E0000C701B6010E94422018160CF05BC2EBA588
:100E1000FCA580819181029709F454C2D1018D9182
:100E20009C911197029709F44DC222853385448520
:100E300055851A966D917D918D919C911D970E947B
:100E40007B1F2B013C01C80117FD0196BC01759564
:100E50006795882777FD8095982F0E94E4209B0155
:100E6000AC01C301B2010E94F22118167CF4B80152
:100E7000882777FD8095982F0E94E4209B01AC0184
:100E8000C301B2010E947B1F2B013C01B80117FF77
:100E900002C06F5F7F4F7595679571956195710978
:100EA000882777FD8095982F0E94E4209B01AC0154
:100EB000C301B2010E94422087FF0FC0B8018827FA
:100EC00077FD8095982F0E94E4209B01AC01C3011F
:100ED000B2010E947C1F2B013C01F101C680D7802A
:100EE000E084F184ABA5BCA516968D909D90AD9045
:100EF000BC901997A5019401C701B6010E947B1F00
:100F00006DA37EA38FA398A72F89388D498D5A8D05
:100F10000E94FD219B01AC01C301B2010E947C1F14
:100F2000B1E0BB8720E030E0A9010E94F221181651
:100F30000CF01B86E1E0EF8720E030E0A901C3015F
:100F4000B2010E94F22118160CF01F86FB852F8536
:100F5000F21709F4B7C1A7019601C501B4010E94B7
:100F60007B1F6B877C878D879E8720E030E0A901FF
:100F70000E94F221181634F06B857C858D859E8544
:100F8000905804C06B857C858D859E850831110540
:100F90002CF020E030E040E85EE304C02BEA3AEABF
:100FA0004AE25EE30E94F22118160CF008C1A50186
:100FB000940169817A818B819C810E94FD216F87D8
:100FC000788B898B9A8BA70196016D817E818F81A9
:100FD00098850E94FD216B8F7C8F8D8F9E8F2D8138
:100FE0003E814F81588569817A818B819C810E94E5
:100FF0007C1F2B013C012B8D3C8D4D8D5E8D6F85B3
:10100000788989899A890E947C1FA30192010E9494
:10101000492069A37AA38BA39CA3A50194016F85A2
:10102000788989899A890E94FD214B015C01A70179
:1010300096016B8D7C8D8D8D9E8D0E94FD219B0177
:10104000AC01C501B4010E947C1F6B017C0129A188
:101050003AA14BA15CA1C301B2010E94FD2129A1CB
:101060003AA14BA15CA10E94FD219B01AC01C701EB
:10107000B6010E947B1F20E030E040E05FE30E9469
:10108000FD2120E030E84BE356E40E94F2211816DF
:101090000CF047C0C9A0DAA0EBA0FCA0ABA5BCA592
:1010A0001696CD92DD92ED92FC921997F101228174
:1010B00033814481558112966D917D918D919C91E2
:1010C00015970E947C1FABA5BCA512966D937D93CE
:1010D0008D939C931597E2E0F0E0ED93FC93D101A2
:1010E0001D921C92F10112821382148215820E94B9
:1010F000071B6B017C012CED35E040E050E064EF14
:1011000071E080E090E00E945F1F6C0D7D1D8E1DE0
:101110009F1DD10156966D937D938D939C93599706
:10112000D1C02DEC3CEC4CE45FE369817A818B818A
:101130009C810E94FD212B853C854D855E850E940A
:10114000FD212F85388949895A890E947C1F2B8D62
:101150003C8D4D8D5E8D0E947C1FA30192010E94EB
:101160004920F10166837783808791872DEC3CECE1
:101170004CE45FE36D817E818F8198850E94FD2123
:101180002DA13EA14FA158A50E94FD212F85388990
:1011900049895A890E947C1F2B8D3C8D4D8D5E8D17
:1011A0000E947C1FA30192010E944920ABA5BCA50F
:1011B00016966D937D938D939C93199783C02D8183
:1011C0003E814F81588569817A818B819C810E9403
:1011D0007C1F2B013C0120E030E040E850E40E94FD
:1011E000F2211816C4F4A3E0CA2ED12CEBA5FCA55D
:1011F000D182C08220E030E040E85FEB228333837D
:10120000448355830E94071BEBA5FCA5668B778B57
:10121000808F918F39C0A501940169817A818B817A
:101220009C810E94FD214B015C01A70196016D810B
:101230007E818F8198850E94FD219B01AC01C501B3
:10124000B4010E947C1FA30192010E944920ABA51A
:10125000BCA516966D937D938D939C931997F10180
:10126000228133814481558112966D917D918D91BA
:101270009C9115970E947C1FABA5BCA512966D93FF
:101280007D938D939C931597F101118210821282A8
:101290001382148215820E94071B6B017C012CEDC6
:1012A00035E040E050E064EF71E080E090E00E94C3
:1012B0005F1F6C0D7D1D8E1D9F1DF101668B778B51
:1012C000808F918F2F8D38A12F5F3F4F38A32F8FA5
:1012D0003AE1230E311C5ECDE9A4FAA4FCA6EBA6EC
:1012E0003ACD212C312C80910A0190910B012816C6
:1012F00039060CF03DC240E060E080E00E944F15EE
:101300002B013C012BED31E03C872B871A8219829F
:101310006101EE24D7FCE094FE2CCD82DE82EF82C8
:10132000F88600910A0110910B01083111051CF09B
:1013300083E090E002C082E090E0C980DA80C816C5
:10134000D9060CF00AC2AB85BC85AD90BC90A11447
:10135000B10409F4F6C16D817E818F8198850E9468
:10136000E4209B01AC01EB85FC8562857385848557
:1013700095850E947B1F6B017C01C80117FD0196BA
:10138000BC0175956795882777FD8095982F0E94F9
:10139000E4209B01AC01C701B6010E94F22118169E
:1013A0007CF4B801882777FD8095982F0E94E4206F
:1013B0009B01AC01C701B6010E947B1F6B017C0140
:1013C000B80117FF02C06F5F7F4F759567957195E4
:1013D00061957109882777FD8095982F0E94E420F8
:1013E0009B01AC01C701B6010E94422087FF0FC0DC
:1013F000B801882777FD8095982F0E94E4209B01F3
:10140000AC01C701B6010E947C1F6B017C0120E08A
:1014100030E0A901C701B6010E94F22118165CF460
:1014200020E030E040E85FE3C701B6010E944220BF
:1014300087FF87C10BC020E030E040E85FEBC701C9
:10144000B6010E94F22118160CF07BC1C50101976C
:1014500020E030E0A901029708F098C0C701B6016A
:101460000E94F22118164CF4A701960160E070E08A
:1014700080E89FE30E947B1F08C020E030E040E846
:101480005FE3C701B6010E947C1F20E030E040EF1F
:1014900051E40E94FD216B017C0120E030E048E432
:1014A00053E4AB85BC8552966D917D918D919C9155
:1014B00055970E9449204B018C012DEC3CEC4CECE3
:1014C0005DE30E94422087FD0FC020E030E040E055
:1014D00050E4B401C8010E94F221181654F480E0CF
:1014E00090E000E010E406C08DEC9CEC0CEC1DE3F9
:1014F00001C0C4019C01A801C701B6010E94FD21E1
:101500000E94B1206B017C017A876987B2E0AB163B
:10151000B10461F4CB0177FD039695958795959578
:101520008795482F60E00E944F1527C020E030E0EB
:1015300040E05FE3AB85BC8512966D917D918D9106
:101540009C9115970E947B1F20E030E04AE253E413
:101550000E94FD2120E030E040E650E40E94492056
:1015600020E030E04AEA52E40E947C1F0E94B12051
:10157000DC01CB016C2D0E944E029B01AC01C3012A
:10158000B2010E94D9022B013C01DBC0C701B601A8
:101590000E94F221181664F420E030E040E05FE39E
:1015A000C701B6010E94422018160CF4CAC00AC036
:1015B00020E030E040E05FEBC701B6010E94F2217D
:1015C00087FDBFC0B3E0AB16B10469F40E94071BEE
:1015D000EB85FC8506891789208D318D601B710B89
:1015E000820B930B45C0F4E0AF16B10409F05EC066
:1015F0000E94071BAB85BC8556960D911D912D91C0
:101600003C915997601B710B820B930B62337105F0
:101610008105910508F42CC10E94071BEB85FC8510
:1016200006891789208D318D601B710B820B930BFE
:10163000643671058105910508F41FC10E94071BDE
:101640008B019C01EB85FC8586899789A08DB18DE6
:101650004CE9C42EDD24DA94ED2CFD2CC81AD90AED
:10166000EA0AFB0AC701B601600F711F821F931FB0
:1016700022E330E040E050E00E942424CA01B90196
:101680000E94E2209B01AC0160E070E080E090E409
:101690000E9460229B01AC0160E070E088EC92E463
:1016A0000E9449200E94B1207A876987E984FA84E0
:1016B0001E141F0414F54985642F842F0E944F15B2
:1016C0009B01AC01C301B2010E94D9022B013C0174
:1016D00020E030E040E85FE3AB85BC8512966D9179
:1016E0007D918D919C9115970E947B1FEB85FC85C8
:1016F000628373838483958324C0AB85BC851196F4
:101700001C921E92FD0112821382148215820E9485
:10171000071B6B017C012CED35E040E050E064EFED
:1017200071E080E090E00E945F1F6C0D7D1D8E1DBA
:101730009F1DAB85BC8556966D937D938D939C9331
:101740005997E981FA813196FA83E9832B853C85A3
:10175000265E3F4F3C872B87E4CDA3019201B10168
:1017600089EB91E00E94EA141FEF211A310ABBCDE8
:1017700089EB91E0AC960FB6F894DEBF0FBECDBFFB
:10178000DF91CF911F910F91FF90EF90DF90CF905D
:10179000BF90AF909F908F907F906F905F904F9091
:1017A0003F902F900C94CE1351824082F301168A01
:1017B000178A108E118E21E931E040E050E062E39B
:1017C00070E080E090E00E945F1F0E94E42020E033
:1017D00030E048EC52E40E944920D30112966D9308
:1017E0007D938D939C93159780910A0190910B01A5
:1017F0009C01442737FD4095542F60E070E0CB01F9
:101800000E945F1F0E94E420F30162877387848730
:10181000958780910A0190910B01D89E4001D99E35
:10182000900C1124FFEF8F1A9F0A9401442737FD73
:101830004095542F1C2DBC011603F001179FF00D8D
:101840001124BF01882777FD8095982F0E945F1F84
:101850000E94E42020E030E040E251E40E94492070
:10186000D30116966D937D938D939C93199781C8A0
:10187000E4E6F0E0FA87E9871ECF21E030E03A871E
:10188000298719CF22E530E048E06CE370E089EB6E
:1018900091E00E94C21469E68AEA91E00C94F21980
:1018A00089EB91E00C9436134F925F926F927F9286
:1018B0008F929F92AF92BF92CF92DF92EF92FF9260
:1018C0000F931F93CF93DF93CDB7DEB7C851D140AD
:1018D0000FB6F894DEBF0FBECDBF9E012F5F3E4F07
:1018E0006901AE014D5F5E4F7A018E010B5F1E4FA5
:1018F0002A5F3F4F4A5F5F4FBE01655F7E4F8AEAB6
:1019000091E00E940B1A80915303811141C0109203
:10191000700310927103109272031092730310926D
:1019200058031092590310925A0310925B031092BD
:101930005C0310925D0310925E0310925F0310929D
:10194000600310926103109262031092630310927D
:10195000540310925503109256031092570310929D
:10196000640310926503109266031092670310924D
:1019700068031092690310926A0310926B0310922D
:101980006C0310926D0310926E0310926F030BC2E2
:10199000C55FDE4F68817981CB50D140882777FDC4
:1019A0008095982F0E94E42020E030E040E858E342
:1019B0000E94FD212B013C01C75FDE4F68817981C8
:1019C000C950D140882777FD8095982F0E94E42048
:1019D00020E030E040E858E30E94FD214B015C012B
:1019E000609368037093690380936A0390936B0319
:1019F000C95FDE4F68817981C750D140882777FD64
:101A00008095982F0E94E42020E030E040E858E3E1
:101A10000E94FD21C35FDE4F688379838A839B83A5
:101A2000CD50D140CB5FDE4F68817981C550D14028
:101A3000882777FD8095982F0E94E4202FE632E1D9
:101A400043E053E40E944920CF5EDE4F68837983F0
:101A50008A839B83C151D140CD5FDE4F68817981FC
:101A6000C350D140882777FD8095982F0E94E420AD
:101A70002FE632E143E053E40E9449206B017C01F0
:101A800060935C0370935D0380935E0390935F03A8
:101A9000CF5FDE4F68817981C150D140882777FDC3
:101AA0008095982F0E94E4202FE632E143E053E432
:101AB0000E94492077FA709477F8709440926C03F2
:101AC00050926D0360926E0370926F03C35FDE4F9E
:101AD000288139814A815B81CD50D1405058C35F04
:101AE000DE4F288339834A835B83CD50D1402093D6
:101AF0006403309365034093660350936703CF5E9E
:101B0000DE4F288139814A815B81C151D1405058D3
:101B1000CF5EDE4F288339834A835B83C151D14036
:101B200020936003309361034093620350936303F7
:101B30009B01AC015058CB5EDE4F288339834A832A
:101B40005B83C551D1402093580330935903409390
:101B50005A0350935B03C301B2010E94F4222B018C
:101B60003C01C501B4010E94F4229B01AC01C301F8
:101B7000B2010E947C1F4B015C01C35FDE4F688194
:101B800079818A819B81CD50D1400E94F4229B01B2
:101B9000AC01C501B4010E947C1F0E94B62220E066
:101BA00030E040E85FE30E947B1F60935403709332
:101BB000550380935603909357032DEC3CEC4CEC6B
:101BC0005DE30E94F22118160CF444C020E030E0DE
:101BD0004AE753E4CF5EDE4F688179818A819B8139
:101BE000C151D1400E9449200E94F4224B015C0166
:101BF00020E030E04AE753E4C701B6010E944920E3
:101C00000E94F4229B01AC01C501B4010E947C1F1B
:101C10006B017C0120E030E04AE753E4CB5EDE4F0D
:101C2000688179818A819B81C551D1400E94492078
:101C30000E94F4229B01AC01C701B6010E947C1FE7
:101C40000E94B6222DEC3CEC4CEC5DE30E94F221AC
:101C500018166CF40E94071B60934F037093500397
:101C6000809351039093520310920C0116C00E946E
:101C7000071BC0904F03D0905003E0905103F090A9
:101C800052036C197D098E099F09693873418105DA
:101C9000910518F081E080930C010E94071BC09011
:101CA000CE01D090CF01E090D001F090D1016C191D
:101CB0007D098E099F09693E73408105910520F0D9
:101CC0001092D3011092D201A090D201B090D30112
:101CD000A0FC29C020E030E045E753E460915803C0
:101CE0007091590380915A0390915B030E94F221F5
:101CF00018160CF058C05FEFA51AB50AB092D301C0
:101D0000A092D2010E94071B6093CE017093CF0175
:101D10008093D0019093D1018091D3018F938091D2
:101D2000D2018F9326C020E030E045E753EC60916C
:101D300058037091590380915A0390915B030E945C
:101D4000422087FF30C08FEFA81AB80AB092D301A3
:101D5000A092D2019FEFC91AD90AE90AF90AC092E2
:101D6000CE01D092CF01E092D001F092D101BF928A
:101D7000AF928FE091E09F938F938E010F5F1F4F83
:101D80001F930F930E941726B8018DE394E00E94E1
:101D90003F018DE394E00E94651C0F900F900F901F
:101DA0000F900F900F90C85EDE4F0FB6F894DEBF15
:101DB0000FBECDBFDF91CF911F910F91FF90EF909C
:101DC000DF90CF90BF90AF909F908F907F906F905B
:101DD0005F904F9008958F929F92AF92BF92CF9253
:101DE000DF92EF92FF924B015C010E94071B6B0197
:101DF0007C01C80CD91CEA1CFB1C0E94071B6C153B
:101E00007D058E059F0580F40E94071BA7019601A2
:101E1000261B370B480B590B243031054105510562
:101E200060F30E94540CE9CFFF90EF90DF90CF90C9
:101E3000BF90AF909F908F900895BF92CF92DF9206
:101E4000EF92FF920F931F93CF93DF937C0101E0FA
:101E500010E0C801877099279C01359527952827A0
:101E6000392720FF03C0FAE0DF2E01C0D12C21FF6B
:101E700003C0EAE0CE2E01C0C12C22FF03C07AE0ED
:101E8000B72E01C0B12CC0E0D0E080910A01909142
:101E90000B01C817D9070CF54B2D6C2D8D2D0E9409
:101EA0004F159B01AC01BE0189EB91E00E94EA1441
:101EB00089EB91E00E94CE1360910A0170910B01B1
:101EC000C7010E94FC2380E090E00E94EB0E80910D
:101ED0000C01882341F02196D8CF0F5F1F4F0131AD
:101EE000110509F0B6CFDF91CF911F910F91FF90AF
:101EF000EF90DF90CF90BF900895CF92DF92EF9256
:101F0000FF920F931F93CF93DF936B017C018A01A4
:101F1000C0E0D0E080910A0190910B01C817D90769
:101F2000E0F4A7019601BE0189EB91E00E94EA145A
:101F300089EB91E00E94CE1360910A0170910B0130
:101F4000C8010E94FC2380E090E00E94EB0E80918B
:101F50000C01882311F02196DDCFDF91CF911F91E5
:101F60000F91FF90EF90DF90CF900895CF92DF9286
:101F7000EF92FF920F931F93CF93DF936B01C0E01B
:101F8000D0E0E82EF12C20910A0130910B01E29E65
:101F9000C001E39E900DF29E900D1124C817D90741
:101FA000B8F5BE0180E090E00E94E22020E030E041
:101FB00040E250E40E94FD210E94B120DC01CB01EF
:101FC0006AE00E944E028B019C0160910A017091AF
:101FD0000B01CE010E94FC23A9019801BC0189EBF1
:101FE00091E00E94EA1489EB91E00E94CE13609187
:101FF0000A0170910B01C6010E94FC2380E090E071
:102000000E94EB0E80910C01882311F02196BBCF2A
:10201000DF91CF911F910F91FF90EF90DF90CF90C4
:1020200008958F929F92AF92BF92CF92DF92EF92DC
:10203000FF920F931F93CF93DF93C82ED12CDC2CEC
:10204000CC24872E912CA12CB12C00E010E00C1593
:102050001D0569F1E12CF12CC0E0D0E060910A018E
:1020600070910B01C617D70798F4C7010E94FC2393
:10207000CB016AE0800F911F0E944E029B01AC01D0
:10208000BE0189EB91E00E94EA142196F394E6CF19
:1020900089EB91E00E94CE13C501B4010E94EB0EC2
:1020A00080910C01882319F00F5F1F4FD0CFDF9173
:1020B000CF911F910F91FF90EF90DF90CF90BF9045
:1020C000AF909F908F9008954F925F926F927F9202
:1020D0008F929F92AF92BF92CF92DF92EF92FF9238
:1020E0000F931F93CF93DF936B017C012A01612C27
:1020F000712C4901A12CB12C6414750409F441C060
:10210000C0E0D0E000E010E080910A0190910B0166
:102110000817190764F4B8016C0F7D1FA701960119
:1021200089EB91E00E94EA140D5F1F4FEDCF89EB20
:1021300091E00E94CE13C501B4010E94EB0E809184
:102140000C018823F1F000E010E080910A019091E9
:102150000B01081719076CF4B8016C0F7D1F20E004
:1021600030E0A90189EB91E00E94EA140D5F1F4F56
:10217000ECCF2196C330D10529F68FEF681A780A83
:10218000BBCFDF91CF911F910F91FF90EF90DF9028
:10219000CF90BF90AF909F908F907F906F905F9007
:1021A0004F9008952F923F924F925F926F927F923D
:1021B0008F929F92AF92BF92CF92DF92EF92FF9257
:1021C0000F931F93CF93DF931C01412C512C612C53
:1021D000712C6B01E12CF12C6214730409F44BC0D7
:1021E0006AE0842D90E00E944E024B015C01C0E049
:1021F000D0E000E010E080910A0190910B010817F7
:10220000190764F4B8016C0F7D1FA501940189EBD7
:1022100091E00E94EA140D5F1F4FEDCF89EB91E032
:102220000E94CE13C701B6010E94EB0E80910C01F3
:10223000882309F100E010E080910A0190910B01E0
:10224000081719076CF4B8016C0F7D1F20E030E00F
:10225000A90189EB91E00E94EA140D5F1F4FECCFBA
:102260002196C330D10529F68FEF681A780A85E0E8
:10227000480E511CB1CFDF91CF911F910F91FF906C
:10228000EF90DF90CF90BF90AF909F908F907F9016
:102290006F905F904F903F902F9008954F925F9274
:1022A0006F927F928F929F92AF92BF92CF92DF9266
:1022B000EF92FF920F931F93CF93DF936C01CC0C9F
:1022C000DD1CC80ED91E00E010E0812C99249394E7
:1022D0002B01612C712C0C151D0509F453C0C0E0B5
:1022E000D0E0A12CB12CE12CF12C60910A0170916D
:1022F0000B01E616F706DCF4C5010E941024CB01A1
:10230000800F911FB4010E9410246AE00E944E02C7
:102310009B01AC01B7016C0F7D1F89EB91E00E941E
:10232000EA1483E0E80EF11C8DEFB81ADECF89EBDA
:1023300091E00E94CE13C301B2010E94EB0E809186
:102340000C018823F9F0E12CF12C80910A01909185
:102350000B01E816F90674F4B7016C0F7D1F20E03D
:1023600030E0A90189EB91E00E94EA1483E0E80ED5
:10237000F11CEBCF2196C330D10509F0B2CF0D5F30
:102380001F4FA9CFDF91CF911F910F91FF90EF9039
:10239000DF90CF90BF90AF909F908F907F906F9085
:1023A0005F904F9008958F929F92AF92BF92CF927D
:1023B000DF92EF92FF920F931F93CF93DF934C0125
:1023C00084E6869F8001879F100D1124C0E0D0E035
:1023D000AA2497FCA094BA2CC017D1070CF050C0C7
:1023E00064E670E080E090E00E943B1F681579058C
:1023F0008A059B05CCF560910A0170910B01882735
:1024000077FD8095982F0E943B1F6B017C0160E057
:1024100071E080E090E00E943B1FDC01CB0164E6AC
:102420000E944E029B01AC01B60189EB91E00E9433
:10243000EA1489EB91E00E94CE136AE070E080E03C
:1024400090E00E94EB0E80910C018823C9F020E0FF
:1024500030E0A901B60189EB91E00E94EA1489EB12
:1024600091E00E94CE130AC06AE070E080E090E044
:102470000E94EB0E80910C01882311F02196ACCFC5
:10248000DF91CF911F910F91FF90EF90DF90CF9050
:10249000BF90AF909F908F9008958091A9018F93E6
:1024A0008091A8018F9389E691E09F938F938FE4A9
:1024B00092E09F938F930E9417266FE472E08DE362
:1024C00094E00E943F018DE394E00E94651C0F9010
:1024D0000F900F900F900F900F90E091A801F09146
:1024E000A9013197EB30F10508F076C0EC5CFF4FA5
:1024F0000C9465248EEE92E00E941D0F67C04AE0A6
:102500006AE00FC06EEE72E08FE00E94B60F40E00E
:1025100060E080E00E944F154EEE52E04EC040E079
:1025200060E08AE03DC060EA7FE085E00E94111033
:102530003DC040E033C040E060E08AE00E944F15BB
:1025400024E630E044E150E00E94641040E06AE09C
:1025500080E00E944F1524E630E044E150E00E9404
:1025600064104AE060E080E00E944F1524E630E00D
:1025700044E150E00E94641064E670E08CE390E077
:102580000E94D21023C04AE060E009C064E670E017
:102590008CE390E00E944E1119C04AE06AE080E0AE
:1025A0000E944F1548EE53E00E947D0F40E060E02E
:1025B00080E00E944F1548EE53E00E947D0F06C058
:1025C0006AE070E084E190E00E94D3118091A8015C
:1025D0009091A901019602C081E090E09093A90139
:1025E0008093A80108958091530381110AC06091DE
:1025F000D40181E068276093D4018DE00E94D31B51
:1026000032C00E94540C2091D2013091D3018091AC
:10261000D5019091D6012730310558F018161906CA
:1026200024F59195819591099093D6018093D501D8
:10263000089597FF10C081E090E09093D6018093B9
:10264000D5010E94071B6093D7017093D801809336
:10265000D9019093DA018091D5019091D60101972B
:1026600011F40C9466030C944D120895CF93DF93EC
:10267000EC0188859985009711F00E9424258E81B0
:1026800087FD05C060E0DF91CF910C949A1BDF912C
:10269000CF910895CF93DF93EC018E8187FD07C022
:1026A00061E00E949A1B60E08E810E94D31B81E052
:1026B0008983DF91CF910895EF92FF920F931F933B
:1026C000CF93DF93EC017B0188859985009711F00A
:1026D0000E9424259D858A85981303C083E090E09D
:1026E00002C084E090E08E9D80018F9D100D9E9D24
:1026F000100D11241D830C83C8010E948C2499871E
:102700008887009741F0A80160E070E00E941026E1
:10271000FB82EA8204C01D821C821B821A82DF9126
:10272000CF911F910F91FF90EF900895FC0121E050
:1027300095858285981320E0CB0136E096958795A4
:102740003A95E1F7482F43704587CB0154E09695C1
:1027500087955A95E1F7382F33703287CB019695DC
:1027600087959695879583708387862F8370848756
:1027700081E06F3F710511F008F080E08083808573
:102780009185892B51F091E0431390E0921729F045
:1027900062817381CF010C945C130895CF92DF9214
:1027A000EF92FF920F931F93CF93DF93CDB7DEB7D6
:1027B00029970FB6F894DEBF0FBECDBF8C01DC01A8
:1027C00018968D919C911997892B09F49AC00E94B3
:1027D000131BF801C684D784E088F1886C197D0941
:1027E0008E099F09623371058105910580F3F89484
:1027F000848195819A838983A085B1857D01EFEFDE
:10280000EE1AFE0A8C918987D8019C9152960D9000
:10281000BC91A02DF8018489992309F42EC09C91C4
:10282000982B98879C91809589238F838F818E83A5
:1028300088E08D8358856F8149853D812E8189810E
:102840009A81F7015C9347FD252F3A952C93262F0B
:1028500039F0441F00C000006C93000000C0F2CFAC
:1028600038E041916C930000019761F7F801B38B58
:10287000A28B49873D832E8338C09C91982B9887E3
:102880009C91809589238F838F818C8388E08B83B3
:1028900058856F8149853B812C8189819A81F70117
:1028A0005C9347FD252F00C000C02C9300C000C0E2
:1028B00000C000C000C06C930000262F3A9541F084
:1028C000441F000000C000C000C000C000C0E8CF2E
:1028D00038E0419100C06C9300C0019709F7F801FE
:1028E000B38BA28B49873B832C839A83898378940B
:1028F0000E94131BD8011E966D937D938D939C931C
:10290000519729960FB6F894DEBF0FBECDBFDF9169
:10291000CF911F910F91FF90EF90DF90CF9008958E
:102920001F93CF93DF93EC01162F8981882331F019
:102930008E8187FD03C060E00E949A1B1E838981FF
:10294000882341F061E0812F0E949A1B60E0812F73
:102950000E94D31B812F90E0FC01E650FE4FE491D2
:10296000F0E0EE0FFF1FE25FFD4F259134913B8BAE
:102970002A8BFC01EA51FE4F84918C8BDF91CF9121
:102980001F910895EF92FF920F931F93CF93DF93C0
:102990001F92CDB7DEB77C018B01FC01118217823B
:1029A0001186108616861786108A118AB901498306
:1029B0000E949613B801C7010E945C134981642FDD
:1029C000C7010F90DF91CF911F910F91FF90EF9072
:1029D0000C949014CF92DF92EF92FF920F931F937B
:1029E000CF93DF93FC01828193816817790708F008
:1029F0004DC0CA01AA27BB27182FC32ED42EE52EFF
:102A0000FF24DC2DC22F0781002361F0809FC001CD
:102A10001124192FC09E60011124DD2D209FC001BB
:102A20001124C92FF5848285A085B185F81208C0CC
:102A3000CB01880F991F860F971F8A0F9B1F17C006
:102A4000CB01880F991F880F991F8A0F9B1F452F55
:102A5000552766277727DC01AF0DB11D002329F02C
:102A6000409F90011124232F01C0242F2C932285F5
:102A7000DC01A20FB11D1C932385DC01A20FB11D47
:102A8000DC932485FC01E20FF11DC083DF91CF911F
:102A90001F910F91FF90EF90DF90CF900895962FA8
:102AA00050E060E070E0592B682BCB01BA0108952B
:102AB0008091A40390E02091A503821B91090895C1
:102AC0002091A5038091A403281750F4E22FF0E091
:102AD000EA55FC4F808190E02F5F2093A503089575
:102AE0008FEF9FEF0895E091A5038091A403E8176D
:102AF00030F4F0E0EA55FC4F808190E008958FEFCC
:102B00009FEF08950895CF92DF92EF92FF920F9377
:102B10001F93CF93DF937C01CB018A012091800327
:102B2000222389F0EB016B01C40ED51ECC15DD0507
:102B300069F06991D701ED91FC910190F081E02D50
:102B4000C7010995F3CF642F0E94E216C801DF91F7
:102B5000CF911F910F91FF90EF90DF90CF9008954C
:102B6000CF93DF931F92CDB7DEB7698320918003A7
:102B70002223D1F020918103203240F021E030E087
:102B8000FC013383228380E090E015C080918203B2
:102B9000E82FF0E0ED57FC4F998190838F5F809391
:102BA00082038093810305C061E0CE0101960E94FB
:102BB000E21681E090E00F90DF91CF910895FC0143
:102BC0001382128248EE53E060E070E04483558344
:102BD000668377838AE791E09183808308951092DA
:102BE000A5031092A40310928203109281030C9407
:102BF0002D16862F413208F040E266EA73E00E940B
:102C00004B161092A5038093A403089521E00C9421
:102C1000F91581E0809380036093A30310928203EF
:102C20001092810308950F93062F21E040918103B4
:102C300063E873E08091A3030E948F1610928203D1
:102C400010928103109280030F91089561E00C941B
:102C5000131684E793E00C94DF151092330481E09F
:102C6000809331041092300461E082E10E94D31B12
:102C700061E083E10E94D31BE9EBF0E080818E7F6D
:102C8000808380818D7F808388E48093B80085E491
:102C90008093BC000895413208F03FC09091330406
:102CA0009111FCCF91E090933304209331042FEFE6
:102CB0002093C60310920B04240F20930A049093D0
:102CC000320490913204880F892B809332048091D2
:102CD0003004813041F410923004809132048093AA
:102CE000BB0085EC01C085EE8093BC00809133046D
:102CF0008130E1F380910B04841710F440910B04B0
:102D00002CE034E0FB01D9018A2F821B841718F4D0
:102D10008D918193F9CF842F089580E008950F93CA
:102D2000413208F046C0909133049111FCCF92E0FB
:102D300090933304009331049FEF9093C603109255
:102D40000B0440930A04FB016CE074E0DB019A2F52
:102D5000961B941718F491919D93F9CF1092320419
:102D600090913204880F892B809332048091300433
:102D7000813041F410923004809132048093BB0082
:102D800085EC01C085EE8093BC00222321F0809168
:102D900033048230E1F38091C6038F3F61F080916C
:102DA000C603803251F08091C603803341F483E042
:102DB00007C081E005C080E003C082E001C084E07C
:102DC0000F910895613298F420913304243089F4EE
:102DD0006093E803FC018AEE93E0DC012A2F281BB4
:102DE000261718F421912D93F9CF80E0089581E002
:102DF000089582E0089585ED8093BC008091BC0029
:102E000084FDFCCF10923304089585EC8093BC00C0
:102E10001092330408951F920F920FB60F9211244F
:102E20002F933F934F935F936F937F938F939F93D2
:102E3000AF93BF93EF93FF938091B900887F803663
:102E400009F49CC068F5883209F45BC090F48031C5
:102E500009F454C038F4882309F4F5C0883009F423
:102E60004DC0F5C0883109F44CC0803209F45DC012
:102E7000EEC0803409F468C048F4803309F455C0CA
:102E8000883309F0E4C08093C603A8C0803509F4F4
:102E90004FC0883509F45DC0883409F0D8C0D5C06A
:102EA000883909F4C6C0A8F4883709F467C038F433
:102EB000883609F463C0803709F460C0C8C0883818
:102EC00009F4B7C0803909F45FC0803809F0BFC089
:102ED0005BC0803B09F485C038F4803A09F466C0D1
:102EE000883A09F47EC0B3C0803C09F4A6C0883C8F
:102EF00009F4A3C0883B09F489C0A9C080913204B9
:102F000010C090910B0480910A04981770F5E0911D
:102F10000B0481E08E0F80930B04F0E0E45FFB4F25
:102F200080818093BB0085EC85C08093C6038DC0F3
:102F3000E0910B0481E08E0F80930B048091BB0025
:102F4000F0E0E45FFB4F808390910B0480910A04D2
:102F50006DC0E0910B0481E08E0F80930B04809193
:102F6000BB00F0E0E45FFB4F80838091310481116E
:102F70006CC081E08093300484EA60C083E0809379
:102F800033041092C703CFCF8091C703803208F07B
:102F900050C0E091C70381E08E0F8093C7038091FA
:102FA000BB00F0E0E853FC4F8083BDCF8091C703A6
:102FB000803230F4E091C703F0E0E853FC4F108218
:102FC0000E94FB166091C70370E0E0912C04F09121
:102FD0002D0488EC93E009951092C7030E94051711
:102FE00036C084E0809333041092E9031092E80322
:102FF000E0912E04F0912F0409958091E80381114E
:1030000005C081E08093E8031092EA03E091E903B0
:1030100081E08E0F8093E903F0E0E651FC4F808160
:103020008093BB009091E9038091E803981708F41E
:103030007ACF85E88093BC000AC085EC8093BC0001
:103040001092330404C01092C6030E94FB16FF9135
:10305000EF91BF91AF919F918F917F916F915F9110
:103060004F913F912F910F900FBE0F901F90189589
:10307000EF92FF920F931F93CF93DF9300D0CDB7C2
:10308000DEB7062F142F682F84E793E029833A8355
:103090000E940916602F84E793E00E94B0152981F1
:1030A000022FE22E3A81F32E8E2D801B811740F4E1
:1030B000F70161917F0184E793E00E94B015F4CF9E
:1030C00084E793E00E94261691E0811190E0892F19
:1030D0000F900F90DF91CF911F910F91FF90EF9084
:1030E0000895CF93DF931F92CDB7DEB749839E013A
:1030F0002F5F3F4F41E00E9438180F90DF91CF9132
:1031000008953F924F925F926F927F928F929F921B
:10311000AF92BF92CF92DF92EF92FF920F931F93E5
:10312000CF93DF9300D000D000D0CDB7DEB7682EAC
:10313000562E742E3A8329830E94071B6B017C0153
:10314000312C412C872D90E09C838B834801A12C4E
:10315000B12C3714B0F5662D84E793E00E94091670
:10316000652D84E793E00E94B01584E793E00E9408
:103170002616662D84E793E00E9409164B815C8138
:10318000431951094132510514F040E250E0662DD7
:1031900084E793E00E94061684E793E00E945815A6
:1031A000892B59F10115110599F10E94071B6C1922
:1031B0007D098E099F09681579058A059B0540F1EF
:1031C0001CC001151105A9F10E94071B6C197D098E
:1031D0008E099F0920E030E060177107820793078E
:1031E00040F1872D90E0242D332727FD30952817B7
:1031F0003907FCF444244A941CC084E793E00E94FD
:103200002616872D90E2971508F480E2380EA1CF9C
:10321000E981FA81E40DF11D47FCFA95FE83ED8307
:1032200084E793E00E946015ED81FE8180834394E2
:10323000B3CF842D26960FB6F894DEBF0FBECDBF58
:10324000DF91CF911F910F91FF90EF90DF90CF9082
:10325000BF90AF909F908F907F906F905F904F90B6
:103260003F9008950F931F9389019A0141E00E94B6
:1032700081181F910F910895CF92DF92EF92FF92E4
:103280000F931F93CF93DF931F92CDB7DEB7C42E5A
:10329000D22E9701AE014F5F5F4F0E9432198823F3
:1032A000F1F04C2D50E04D1951094F5F5F4F61E037
:1032B00070E002C0660F771FDA94E2F7615071097F
:1032C000042E01C0660F0A94EAF72981262330E014
:1032D00002C0359527954A95E2F7F80120830F90B3
:1032E000DF91CF911F910F91FF90EF90DF90CF90E2
:1032F0000895EF92FF920F931F93CF93DF931F9246
:10330000CDB7DEB7182F062FF42EE22E20910D0137
:1033100030910E01AE014F5F5F4F0E9432198981DB
:1033200021E030E00F2C01C0220F0A94EAF7EE20D2
:1033300019F0482F422B03C0422F40954823498360
:10334000602F812F0E9471180F90DF91CF911F91F4
:103350000F91FF90EF900895DF92EF92FF920F93FD
:103360001F93CF93DF931F92CDB7DEB7F82EE62ED3
:10337000D42E122F20910D0130910E01AE014F5F1E
:103380005F4F0E943219882319F14D2D50E0411BE7
:1033900051094F5F5F4FE1E0F0E002C0EE0FFF1F09
:1033A0001A95E2F73197042E01C0EE0F0A94EAF75E
:1033B00001C0000F4A95EAF74E2F409589814823B6
:1033C000E0234E2B49836E2D8F2D0E94711801C072
:1033D00080E00F90DF91CF911F910F91FF90EF90C0
:1033E000DF900895FC01608308950F93062F22E07B
:1033F00044E06BE1FC0180810E94AC190F910895BB
:103400000F93062F22E044E06CE1FC0180810E94D2
:10341000AC190F9108954F925F926F927F928F92A5
:103420009F92AF92BF92CF92DF92EF92FF920F9353
:103430001F93CF93DF93EC015B013A01490128010F
:1034400000910D0110910E019C012F5F3F4F4EE046
:103450006BE388810E948118898190E0982F8827EA
:103460002A81822BF501918380838B8190E0982FB4
:1034700088272C81822BF301918380838D8190E0BA
:10348000982F88272E81822BF40191838083898550
:1034900090E0982F88272A85822BF20191838083E0
:1034A0008B8590E0982F88272C85822BF7019183BC
:1034B00080838D8590E0982F88272E85822BF601BA
:1034C00091838083DF91CF911F910F91FF90EF90B7
:1034D000DF90CF90BF90AF909F908F907F906F9034
:1034E0005F904F900895262F46E06BE6FC018081A7
:1034F0000C9479190F93062F23E042E06BE6FC0150
:1035000080810E94AC190F910895CF93DF93EC0155
:1035100061E00E947A1A60E0CE010E94F51960E035
:10352000CE010E94001A60E0CE01DF91CF910C9491
:10353000731AEF92FF920F931F93CF93DF93EC01D7
:10354000E0900D01F0900E018C010F5F1F4F26E0FF
:1035500046E065E788810E943C198981DF91CF911F
:103560001F910F91FF90EF9008950E94991A91E09A
:10357000843309F090E0892F08951F920F920FB6BF
:103580000F9211242F933F938F939F93AF93BF93E9
:103590008091350490913604A0913704B09138049D
:1035A0003091340423E0230F2D3720F40196A11D20
:1035B000B11D05C026E8230F0296A11DB11D209361
:1035C00034048093350490933604A0933704B09369
:1035D00038048091390490913A04A0913B04B09151
:1035E0003C040196A11DB11D8093390490933A04C7
:1035F000A0933B04B0933C04BF91AF919F918F91F6
:103600003F912F910F900FBE0F901F9018952FB7DD
:10361000F89460913504709136048091370490914C
:1036200038042FBF08953FB7F894809139049091E2
:103630003A04A0913B04B0913C0426B5A89B05C078
:103640002F3F19F00196A11DB11D3FBF6627782FAE
:10365000892F9A2F620F711D811D911D42E0660F07
:10366000771F881F991F4A95D1F70895789484B5DC
:10367000826084BD84B5816084BD85B5826085BD6E
:1036800085B5816085BDEEE6F0E080818160808354
:10369000E1E8F0E010828081826080838081816037
:1036A0008083E0E8F0E0808181608083E1EBF0E0FE
:1036B000808184608083E0EBF0E0808181608083A2
:1036C000EAE7F0E08081846080838081826080838B
:1036D0008081816080838081806880831092C100B6
:1036E0000895833081F028F4813099F08230A1F080
:1036F00008958730A9F08830B9F08430D1F48091F2
:1037000080008F7D03C0809180008F778093800040
:10371000089584B58F7702C084B58F7D84BD0895E8
:103720008091B0008F7703C08091B0008F7D80932F
:10373000B0000895CF93DF9390E0FC01EA51FE4F73
:103740002491FC01E650FE4F8491882349F190E0DA
:10375000880F991FFC01E85EFD4FA591B491825F2F
:103760009D4FFC01C591D4919FB7611108C0F89499
:103770008C91209582238C93888182230AC06230A9
:1037800051F4F8948C91322F309583238C93888157
:10379000822B888304C0F8948C91822B8C939FBFDA
:1037A000DF91CF9108950F931F93CF93DF931F92D3
:1037B000CDB7DEB7282F30E0F901EE52FE4F8491ED
:1037C000F901EA51FE4F1491F901E650FE4F0491C0
:1037D0000023C9F0882321F069830E94711B69814D
:1037E000E02FF0E0EE0FFF1FE25FFD4FA591B491D7
:1037F0009FB7F8948C91611103C01095812301C08B
:10380000812B8C939FBF0F90DF91CF911F910F91D0
:103810000895FC01818D228D90E0805C9F4F821B7A
:1038200091098F7399270895FC01918D828D9817C6
:1038300031F0828DE80FF11D858D90E008958FEFB6
:103840009FEF0895FC01918D828D981761F0828D14
:10385000DF01A80FB11D5D968C91928D9F5F9F73C4
:10386000928F90E008958FEF9FEF089586EA9DE193
:10387000892B49F080E090E0892B29F00E94A61D59
:1038800081110C9400000895FC01848DDF01A80FC4
:10389000B11DA35ABF4F2C91848D90E001968F7378
:1038A0009927848FA689B7892C93A089B1898C9197
:1038B00080648C93938D848D981306C00288F3895D
:1038C000E02D80818F7D80830895CF93DF93EC017D
:1038D000888D8823C9F0EA89FB89808185FD05C030
:1038E000A889B9898C9186FD0FC00FB607FCF5CF6A
:1038F000808185FFF2CFA889B9898C9185FFEDCFB2
:10390000CE010E94441CE7CFDF91CF910895CF9262
:10391000DF92FF920F931F93CF93DF931F92CDB748
:10392000DEB76C0181E0D60158968C9358975B9670
:103930009C915B975C968C915C97981307C050960E
:10394000ED91FC915197808185FD2EC0F601038D8C
:1039500010E00F5F1F4F0F731127F02EF601848DBB
:10396000F81211C00FB607FCF9CFD6015096ED91B1
:10397000FC915197808185FFF1CFC60169830E9438
:10398000441C6981EBCF838DE80FF11DE35AFF4F93
:103990006083D6015B960C935B975296ED91FC91F8
:1039A0005397808180620CC0D6015696ED91FC91B0
:1039B000579760835096ED91FC9151978081806478
:1039C000808381E090E00F90DF91CF911F910F9164
:1039D000FF90DF90CF900895BF92CF92DF92EF9249
:1039E000FF92CF93DF93EC016A017B01B22EE8894D
:1039F000F98982E08083411581EE580761057105E0
:103A0000A1F060E079E08DE390E0A70196010E94CB
:103A1000242421503109410951095695479537957C
:103A20002795211580E1380798F0E889F9891082F7
:103A300060E874E88EE190E0A70196010E942424DA
:103A400021503109410951095695479537952795D8
:103A5000EC85FD853083EE85FF852083188EEC890B
:103A6000FD89B082EA89FB89808180618083EA894F
:103A7000FB89808188608083EA89FB8980818068F6
:103A80008083EA89FB8980818F7D8083DF91CF915C
:103A9000FF90EF90DF90CF90BF9008951F920F920C
:103AA0000FB60F9211242F938F939F93EF93FF9351
:103AB000E0914D04F0914E048081E0915304F09127
:103AC000540482FD12C09081809156048F5F8F73E1
:103AD00020915704821751F0E0915604F0E0E35C26
:103AE000FB4F958F8093560401C08081FF91EF9129
:103AF0009F918F912F910F900FBE0F901F9018954F
:103B00001F920F920FB60F9211242F933F934F9352
:103B10005F936F937F938F939F93AF93BF93EF9335
:103B2000FF938DE394E00E94441CFF91EF91BF91BD
:103B3000AF919F918F917F916F915F914F913F9145
:103B40002F910F900FBE0F901F9018958DE394E06A
:103B50000E94091C21E0892B09F420E0822F08959E
:103B60001092400410923F0488EE93E0A0E0B0E091
:103B70008093410490934204A0934304B09344047F
:103B80008AE891E090933E0480933D0485EC90E0B8
:103B900090934A048093490484EC90E090934C0401
:103BA00080934B0480EC90E090934E0480934D04FE
:103BB00081EC90E09093500480934F0482EC90E06D
:103BC000909352048093510486EC90E090935404B7
:103BD0008093530410925604109257041092580484
:103BE00010925904089508950E94361B0E94F31DF7
:103BF0000E945501C6E3DCE10E94F3122097E1F335
:103C00000E94361CF9CFCF92DF92EF92FF920F9372
:103C10001F93CF93DF936C017A01EB01E60EF71E41
:103C200000E010E0CE15DF0561F06991D601ED915D
:103C3000FC910190F081E02DC6010995080F191F34
:103C4000F1CFC801DF91CF911F910F91FF90EF90BD
:103C5000DF90CF900895EF92FF920F931F93CF9331
:103C6000DF938C01FB01C0E0D0E064917F018FEF16
:103C7000E81AF80A662361F0D801ED91FC910190F1
:103C8000F081E02DC8010995C80FD91FF701EDCFCC
:103C9000CE01DF91CF911F910F91FF90EF9008958A
:103CA000DC01ED91FC910190F081E02D099466E931
:103CB00071E00C943F010F931F93CF93DF93EC01BE
:103CC0000E942B1E8C01CE010E94571E800F911F57
:103CD000DF91CF911F910F9108958F929F92AF9294
:103CE000BF92CF92DF92EF92FF920F931F93CF93E9
:103CF000DF93CDB7DEB7A1970FB6F894DEBF0FBE46
:103D0000CDBF7C01C42EE52FCB01D22E19A221E01C
:103D10002D1510F02AE0D22E8E010F5D1F4F8D2C35
:103D2000912CA12CB12C6C2D7E2FA50194010E9409
:103D300024248C2DD29E80191124015011098A301F
:103D400014F4805D01C0895CF80180832115310580
:103D50004105510521F0C22EE32FCA01E4CFB8017D
:103D6000C7010E943F01A1960FB6F894DEBF0FBEB7
:103D7000CDBFDF91CF911F910F91FF90EF90DF901A
:103D8000CF90BF90AF909F908F900895CF92DF9289
:103D9000EF92FF920F931F93CF93DF93EC016A0191
:103DA0007B012115310579F4E881F9810190F081D9
:103DB000E02D642FDF91CF911F910F91FF90EF9035
:103DC000DF90CF9009942A303105E9F477FF1AC0CB
:103DD0006DE20E94501E8C0144275527BA014C19F0
:103DE0005D096E097F092AE0CE010E946D1E800FD9
:103DF000911FDF91CF911F910F91FF90EF90DF9076
:103E0000CF9008952AE0B701A601CE01DF91CF91AE
:103E10001F910F91FF90EF90DF90CF900C946D1E4B
:103E20000F931F93CF93DF93EC019A01AB016627A9
:103E300057FD6095762F0E94C61E8C01CE010E9410
:103E4000571E800F911FDF91CF911F910F91089501
:103E50002115310541F4DC01ED91FC910190F081D7
:103E6000E02D642F09940C946D1E9A01AB0160E063
:103E700070E00C94281FCF93DF9300D000D0CDB713
:103E8000DEB79B01AC01611571058105910569F0F3
:103E900069833A834B835C830E94022629813A819D
:103EA0004B815C810E94462403C060E070E0CB013E
:103EB0000F900F900F900F90DF91CF910895CF92B8
:103EC000DF92EF92FF926B017C0162177307840708
:103ED000950764F4CA01B9016C197D098E099F091F
:103EE0000E943B1F6C0D7D1D8E1D9F1DFF90EF904E
:103EF000DF90CF9008955058BB27AA270ED027C235
:103F0000F0D130F0F5D120F031F49F3F11F41EF4E0
:103F1000C0C10EF4E095E7FBB6C1E92F3AD280F3B9
:103F2000BA17620773078407950718F071F49EF5B6
:103F300052C20EF4E0950B2EBA2FA02D0B01B90141
:103F400090010C01CA01A0011124FF27591B99F00F
:103F5000593F50F4503E68F11A16F040A22F232F1B
:103F6000342F4427585FF3CF469537952795A7956B
:103F7000F0405395C9F77EF41F16BA0B620B730B12
:103F8000840BBAF09150A1F0FF0FBB1F661F771F83
:103F9000881FC2F70EC0BA0F621F731F841F48F438
:103FA000879577956795B795F7959E3F08F0B3CFBE
:103FB0009395880F08F09927EE0F979587950895A8
:103FC00090D158F080E891E009F49EEF91D128F06B
:103FD00040E851E059F45EEF09C05BC1FCC1E92F34
:103FE000E078D7D168F3092E052AC1F326173707E1
:103FF0004807590738F00E2E07F8E02569F0E0254C
:10400000E0640AC0EF6307F8009407FADB01B90126
:104010009D01DC01CA01AD01EF934AD098D10AD0CD
:104020005F91552331F02BED3FE049E450FD49EC21
:1040300063CF0895DF93DD27B92FBF7740E85FE3B3
:104040001616170648075B0710F4D92FCFD19F9398
:104050008F937F936F93C8D2EEE7F0E01DD177D1B5
:104060002F913F914F915F91D4D1DD2349F090582A
:10407000A2EA2AED3FE049EC5FE3D0785D274DDF0F
:10408000DF9165C1DCD008F481E0089539D1E39572
:104090006FC10CD05CC12CD140F023D130F021F4A1
:1040A0005F3F19F0F0C0511197C1F3C072D198F37E
:1040B0009923C9F35523B1F3951B550BBB27AA27A9
:1040C00062177307840738F09F5F5F4F220F331F1B
:1040D000441FAA1FA9F333D00E2E3AF0E0E830D0E7
:1040E00091505040E695001CCAF729D0FE2F27D0EA
:1040F000660F771F881FBB1F261737074807AB07B8
:10410000B0E809F0BB0B802DBF01FF2793585F4F2C
:104110002AF09E3F510568F0B6C05EC15F3FECF3E8
:10412000983EDCF3869577956795B795F7959F5FF1
:10413000C9F7880F911D9695879597F90895E1E045
:10414000660F771F881FBB1F621773078407BA07A4
:1041500020F0621B730B840BBA0BEE1F88F7E095FF
:10416000089504D06894B11137C108951AD188F028
:104170009F5790F0B92F9927B751A0F0D1F0660F53
:10418000771F881F991F1AF0BA95C9F712C0B1306E
:1041900081F021D1B1E008951EC1672F782F8827C3
:1041A000B85F39F0B93FCCF3869577956795B395AD
:1041B000D9F73EF490958095709561957F4F8F4F1C
:1041C0009F4F0895E89409C097FB3EF49095809521
:1041D000709561957F4F8F4F9F4F9923A9F0F92FCD
:1041E00096E9BB279395F695879577956795B7954B
:1041F000F111F8CFFAF4BB0F11F460FF1BC06F5F31
:104200007F4F8F4F9F4F16C0882311F096E911C042
:10421000772321F09EE8872F762F05C0662371F063
:1042200096E8862F70E060E02AF09A95660F771F77
:10423000881FDAF7880F9695879597F90895990F53
:104240000008550FAA0BE0E8FEEF16161706E80760
:10425000F907C0F012161306E407F50798F0621B81
:10426000730B840B950B39F40A2661F0232B242B56
:10427000252B21F408950A2609F4A140A6958FEF75
:10428000811D811D089597F99F6780E870E060E0C7
:1042900008959FEF80EC0895DF93CF931F930F93C2
:1042A000FF92EF92DF927B018C01689405C0DA2EB9
:1042B000EF01AFD0FE01E894A5912591359145918C
:1042C0005591AEF3EF0129DEFE019701A801DA94C2
:1042D00079F7DF90EF90FF900F911F91CF91DF91D1
:1042E000089500240A94161617061806090608955C
:1042F00000240A9412161306140605060895C9CF61
:1043000050D0E8F3E894E0E0BB279F57F0F02AEDA7
:104310003FE049EC06C0EE0FBB0F661F771F881FFA
:1043200028F0B23A62077307840728F0B25A620B8A
:10433000730B840BE3959A9572F7803830F49A9555
:10434000BB0F661F771F881FD2F7904883C1092EC5
:104350000394000C11F4882352F0BB0F40F4BF2BE0
:1043600011F460FF04C06F5F7F4F8F4F9F4F089520
:10437000EF93E0FF06C0A2EA2AED3FE049EC5FEBD5
:10438000CCDDE5DF0F90039401FC9058EBEAF0E000
:1043900074C157FD9058440F551F59F05F3F71F09D
:1043A0004795880F97FB991F61F09F3F79F087959C
:1043B0000895121613061406551FF2CF4695F1DF25
:1043C00008C0161617061806991FF1CF86957105B5
:1043D000610508940895E894BB2766277727CB01E9
:1043E00097F908952CDF08F48FEF08959B01AC0135
:1043F00060E070E080E89FE34CCE0BD0A8CF71DF87
:1044000028F076DF18F0952309F03DCF42CF112434
:10441000E3CFBFDFA0F3959FD1F3950F50E0551F79
:10442000629FF001729FBB27F00DB11D639FAA2709
:10443000F00DB11DAA1F649F6627B00DA11D661F58
:10444000829F2227B00DA11D621F739FB00DA11D79
:10445000621F839FA00D611D221F749F3327A00D33
:10446000611D231F849F600D211D822F762F6A2FCF
:1044700011249F5750408AF0E1F088234AF0EE0F54
:10448000FF1FBB1F661F771F881F91505040A9F761
:104490009E3F510570F0F7CE9FCF5F3FECF3983E03
:1044A000DCF3869577956795B795F795E7959F5FC8
:1044B000C1F7FE2B880F911D9695879597F9089562
:1044C000FA01EE0FFF1F30962105310599F16115B4
:1044D000710561F48038BFE39B0749F16894903817
:1044E000810561F08038BFEF9B0741F0992342F5C9
:1044F000FF3FE1053105210511F1E8940894E795A6
:10450000D901AA2329F4AB2FBE2FF85FD0F310C036
:10451000FF5F70F4A695E0F7F73950F019F0FF3A15
:1045200038F49F779F930CD00F9007FC9058089514
:104530003EF0AFCE60E070E080E89FE308954FE783
:104540009F775F934F933F932F93E3D02F913F91AA
:104550004F915F9152DF50C09F93D2DE0F9007FCC6
:10456000EE5F06CF11F40EF494CE72C01ADFD0F3D2
:104570009923D9F3CEF39F57550B87FF77D00024AB
:10458000A0E640EA900180585695979528F4805C03
:10459000660F771F881F20F026173707480730F46B
:1045A000621B730B840B202931294A2BA695179483
:1045B0000794202531254A2758F7660F771F881F53
:1045C00020F026173707480730F4620B730B840B73
:1045D000200D311D411DA09581F7B901842F9158FF
:1045E000880F9695879508959B01AC0106CF19F425
:1045F0000EF049CEF0CE4DCED4DEC8F39638C0F7DB
:1046000007F80F92E8942BE33AEA48EB5FE703DF01
:104610000F920F920F924DB75EB70F92BAD0E9EC9E
:10462000F0E03ADE4F915F91EF91FF91E595EE1F3B
:10463000FF1F49F0FE57E0684427EE0F441FFA952C
:10464000E1F74195550B2CD00F9007FECFCE089582
:104650009F3F31F0915020F4879577956795B795F6
:10466000880F911D9695879597F908959150504020
:10467000660F771F881FD2F708959F938F937F93BC
:104680006F93FF93EF939B01AC01B7DEEF91FF9126
:1046900003DE2F913F914F915F91AFCEF4CDD8CFF4
:1046A00080DEE8F39923D9F3940F511DBBF39150A9
:1046B000504094F059F0882332F0660F771F881F1E
:1046C00091505040C1F79E3F510544F7880F911D0E
:1046D0009695879597F908955F3FACF0983E9CF0CA
:1046E000BB27869577956795B79508F4B160939544
:1046F000C1F7BB0F58F711F460FFE8CF6F5F7F4F32
:104700008F4F9F4FE3CF68CE0EF0A2CFC2CD6894FB
:10471000BACD47DEC8F39923D1F3C6F3DF93CF9325
:104720001F930F93FF92C92FDD2788232AF021972B
:10473000660F771F881FDAF720E030E040E85FEB74
:104740009FE3883920F0803E30F021968F77D4DBCC
:10475000E1EFF0E003C0D0DBEEE1F1E09DDD8B01A5
:10476000BE01EC01FB2E6F5771097595771F880B01
:10477000990B2ADD28E132E741E35FE34ADEAF2D02
:104780009801AE01FF900F911F91CF91DF91C5DB92
:10479000DECDFA01DC01AA0FBB1F9B01AC01BF57A4
:1047A00028F422273327442750781FC0B75188F4B4
:1047B000AB2F0024469537952795011CA395D2F37E
:1047C000002069F0220F331F441FB395DAF30DD098
:1047D00092CB61307105A0E88A07B94630F49B019D
:1047E000AC016627772788279078309621F02083C0
:1047F0003183428353830895AA1BBB1B51E107C039
:10480000AA1FBB1FA617B70710F0A61BB70B881F60
:10481000991F5A95A9F780959095BC01CD010895EF
:1048200097FB072E16F4009407D077FD09D00E945D
:10483000FC2307FC05D03EF4909581959F4F089589
:10484000709561957F4F0895A1E21A2EAA1BBB1B9C
:10485000FD010DC0AA1FBB1FEE1FFF1FA217B3074C
:10486000E407F50720F0A21BB30BE40BF50B661F62
:10487000771F881F991F1A9469F760957095809526
:1048800090959B01AC01BD01CF010895052E97FBCA
:104890001EF400940E945D2457FD07D00E9424243A
:1048A00007FC03D04EF40C945D2450954095309550
:1048B00021953F4F4F4F5F4F08959095809570958C
:1048C00061957F4F8F4F9F4F0895EE0FFF1F05900B
:1048D000F491E02D0994A29FB001B39FC001A39F62
:1048E000700D811D1124911DB29F700D811D112429
:1048F000911D08950E946B24B7FF0895821B930BAE
:1049000008950E946B24A59F900DB49F900DA49FC5
:10491000800D911D11240895CF93DF93823091056E
:1049200010F482E090E0E091DC04F091DD0420E0FE
:1049300030E0A0E0B0E0309739F140815181481774
:104940005907B8F04817590771F48281938110977D
:1049500029F013969C938E9312972CC09093DD04AC
:104960008093DC0427C02115310531F0421753072D
:1049700018F0A901DB0101C0EF019A01BD01DF01BF
:104980000280F381E02DD7CF21153105F9F0281BE6
:10499000390B2430310580F48A819B8161157105C2
:1049A00021F0FB019383828304C09093DD04809304
:1049B000DC04FE01329644C0FE01E20FF31F819336
:1049C000919322503109398328833AC02091DA0427
:1049D0003091DB04232B41F420910201309103013B
:1049E0003093DB042093DA0420910001309101011F
:1049F0002115310541F42DB73EB740910401509186
:104A00000501241B350BE091DA04F091DB04E21779
:104A1000F307A0F42E1B3F0B2817390778F0AC01E1
:104A20004E5F5F4F2417350748F04E0F5F1F5093BE
:104A3000DB044093DA048193919302C0E0E0F0E05C
:104A4000CF01DF91CF910895CF93DF93009709F4C1
:104A500087C0FC01329713821282C091DC04D0918E
:104A6000DD04209781F420813181280F391F809146
:104A7000DA049091DB048217930779F5F093DB0455
:104A8000E093DA046DC0DE0120E030E0AE17BF072E
:104A900050F412964D915C9113979D01411551056B
:104AA00009F1DA01F3CFB383A28340815181840FEE
:104AB000951F8A179B0771F48D919C911197840F14
:104AC000951F02969183808312968D919C911397E6
:104AD000938382832115310529F4F093DD04E0935B
:104AE000DC043EC0D9011396FC93EE9312974D91CE
:104AF0005D91A40FB51FEA17FB0779F480819181BE
:104B0000840F951F0296D90111969C938E938281F2
:104B1000938113969C938E931297E0E0F0E08A8144
:104B20009B81009719F0FE01EC01F9CFCE010296AE
:104B300028813981820F931F2091DA043091DB04A0
:104B40002817390769F4309729F41092DD04109280
:104B5000DC0402C013821282D093DB04C093DA0417
:104B6000DF91CF9108958F929F92AF92BF92CF9293
:104B7000DF92EF92FF92CF93DF93EC01688179810E
:104B80008A819B81611571058105910521F464E29B
:104B900079ED8BE597E02DE133EF41E050E00E94A5
:104BA000462449015A019B01AC01A7EAB1E40E94E5
:104BB00081246B017C01ACEEB4EFA50194010E944D
:104BC000B428C60ED71EE81EF91EF7FE06C081E007
:104BD000C81AD108E10880E8F80AC882D982EA82B6
:104BE000FB82C701B6019F77DF91CF91FF90EF90D5
:104BF000DF90CF90BF90AF909F908F9008950E94CC
:104C0000B325089586E091E00E94B325089560934E
:104C1000060170930701809308019093090108959C
:104C2000DC0101C06D9341505040E0F70895AEE0C3
:104C3000B0E0EDE1F6E20C94C7280D891E8986E00C
:104C40008C831A8309838FEF9FE79E838D83AE0148
:104C5000475E5F4F6F89788DCE0101960E9439269D
:104C6000EF81F885E00FF11F10822E96E4E00C949E
:104C7000E328ACE0B0E0EFE3F6E20C94B9287C0165
:104C80006B018A01FC0117821682838181FFBDC1FD
:104C9000CE0101964C01F7019381F60193FD8591B8
:104CA00093FF81916F01882309F4ABC1853239F4F8
:104CB00093FD859193FF81916F01853229F4B701AE
:104CC00090E00E942128E7CF512C312C20E02032A7
:104CD000A0F48B3269F030F4803259F0833269F4F9
:104CE00020612CC08D3239F0803339F4216026C028
:104CF0002260246023C0286021C027FD27C030ED3A
:104D0000380F3A3078F426FF06C0FAE05F9E300D87
:104D10001124532E13C08AE0389E300D1124332EF7
:104D200020620CC08E3221F426FD6BC1206406C0C7
:104D30008C3611F4206802C0883641F4F60193FDE8
:104D4000859193FF81916F018111C1CF982F9F7D34
:104D50009554933028F40C5F1F4FFFE3F9830DC087
:104D6000833631F0833771F0833509F05BC022C0A0
:104D7000F801808189830E5F1F4F44244394512C96
:104D8000540115C03801F2E06F0E711CF801A080CB
:104D9000B18026FF03C0652D70E002C06FEF7FEF8A
:104DA000C5012C870E9416282C0183012C852F77A2
:104DB000222E17C03801F2E06F0E711CF801A0809E
:104DC000B18026FF03C0652D70E002C06FEF7FEF5A
:104DD000C5012C870E940B282C012C852068222ECF
:104DE000830123FC1BC0832D90E048165906B0F4C4
:104DF000B70180E290E00E9421283A94F4CFF501B7
:104E000027FC859127FE81915F01B70190E00E9408
:104E1000212831103A94F1E04F1A510841145104FD
:104E200071F7E5C0843611F0893639F5F80127FFAE
:104E300007C060817181828193810C5F1F4F08C020
:104E400060817181882777FD8095982F0E5F1F4FB5
:104E50002F76B22E97FF09C0909580957095619539
:104E60007F4F8F4F9F4F2068B22E2AE030E0A40181
:104E70000E945328A82EA81844C0853729F42F7EF5
:104E8000B22E2AE030E025C0F22FF97FBF2E8F36F8
:104E9000C1F018F4883579F0B4C0803719F088373C
:104EA00021F0AFC02F2F2061B22EB4FE0DC08B2D8C
:104EB0008460B82E09C024FF0AC09F2F9660B92EC7
:104EC00006C028E030E005C020E130E002C020E16B
:104ED00032E0F801B7FE07C0608171818281938161
:104EE0000C5F1F4F06C06081718180E090E00E5F13
:104EF0001F4FA4010E945328A82EA818FB2DFF774E
:104F0000BF2EB6FE0BC02B2D2E7FA51450F4B4FE81
:104F10000AC0B2FC08C02B2D2E7E05C07A2C2B2D8A
:104F200003C07A2C01C0752C24FF0DC0FE01EA0DD0
:104F3000F11D8081803311F4297E09C022FF06C053
:104F40007394739404C0822F867809F0739423FDC0
:104F500013C020FF06C05A2C731418F4530C5718B2
:104F6000732C731468F4B70180E290E02C870E94E0
:104F7000212873942C85F5CF731410F4371801C0D1
:104F8000312C24FF12C0B70180E390E02C870E94EF
:104F900021282C8522FF17C021FF03C088E590E05F
:104FA00002C088E790E0B7010CC0822F867859F0E4
:104FB00021FD02C080E201C08BE227FD8DE2B70136
:104FC00090E00E942128A51438F4B70180E390E016
:104FD0000E9421285A94F7CFAA94F401EA0DF11DFA
:104FE0008081B70190E00E942128A110F5CF3320E5
:104FF00009F451CEB70180E290E00E9421283A9452
:10500000F6CFF7018681978102C08FEF9FEF2C9634
:10501000E2E10C94D528FC0105906150704001102C
:10502000D8F7809590958E0F9F1F0895FC016150D1
:10503000704001900110D8F7809590958E0F9F1FBA
:1050400008950F931F93CF93DF93182F092FEB0130
:105050008B8181FD03C08FEF9FEF20C082FF10C0C6
:105060004E815F812C813D81421753077CF4E8819A
:10507000F9819F012F5F3F4F39832883108306C03A
:10508000E885F985812F0995892B29F72E813F81A4
:105090002F5F3F4F3F832E83812F902FDF91CF9142
:1050A0001F910F910895FA01AA27283051F120315C
:1050B00081F1E8946F936E7F6E5F7F4F8F4F9F4FAC
:1050C000AF4FB1E03ED0B4E03CD0670F781F891FEE
:1050D0009A1FA11D680F791F8A1F911DA11D6A0FBC
:1050E000711D811D911DA11D20D009F468943F916F
:1050F0002AE0269F11243019305D3193DEF6CF016E
:105100000895462F4770405D4193B3E00FD0C9F733
:10511000F6CF462F4F70405D4A3318F0495D31FDA0
:105120004052419302D0A9F7EACFB4E0A6959795F3
:10513000879577956795BA95C9F7009761057105C9
:1051400008959B01AC010A2E069457954795379513
:105150002795BA95C9F7620F731F841F951FA01D6D
:105160000895B7FF0C9481240E948124821B930B25
:1051700008952F923F924F925F926F927F928F92FB
:105180009F92AF92BF92CF92DF92EF92FF920F93D6
:105190001F93CF93DF93CDB7DEB7CA1BDB0B0FB6E0
:1051A000F894DEBF0FBECDBF09942A88398848889D
:1051B0005F846E847D848C849B84AA84B984C88433
:1051C000DF80EE80FD800C811B81AA81B981CE0F2A
:1051D000D11D0FB6F894DEBF0FBECDBFED0108950F
:1051E00012E0C8E2D2E004C0FE010E9467242296C9
:0A51F000CA32D107C9F7F894FFCFC7
:1051FA000000DE048000010000003C0001E80374A6
:10520A0077697374436F756E74203D202533640A81
:10521A0000536176656420746F20454550524F4DA6
:10522A003A2025346420253464202534640A004554
:10523A004550524F4D20636F6E7461696E733A2008
:10524A00253464202534642025346420002D2072FE
:10525A006573746F7265640A005061747465726E66
:10526A00202532640A0000000000B0158315581585
:10527A0060157315821500000000871C031E091CA7
:10528A00221C141C651C0D0A006E616E00696E6694
:08529A00006F7666002E000093
:00000001FF
